:020000040800F2
:10000000200600200101000857150008A51200086D
:100010005515000825060008B72400080000000058
:10002000000000000000000000000000391A000875
:10003000190E00080000000011170008E121000857
:100040001B0100081B0100081B0100081B01000820
:100050001B0100081B0100081B0100081B01000810
:100060001B0100081B0100081B010008AD0A000865
:100070001B0100081B0100081B0100081B010008F0
:100080001B0100081B0100081B0100081B010008E0
:10009000492400081B0100081B010008490E000844
:1000A0001B0100081B0100081B0100081B010008C0
:1000B0001B0100081B010008412200081B01000869
:1000C0001B0100081B0100081B0100081B010008A0
:1000D0001B0100081B0100081B0100081B01000890
:1000E000450E00081B0100085D220008DFF80CD057
:1000F00000F0F8F9004800478D2500082006002090
:100100000648804706480047FEE7FEE7FEE7FEE7B1
:10011000FEE7FEE7FEE7FEE7FEE7FEE7F121000867
:10012000ED0000082DE9F05F0546002092469B4651
:1001300088460646814640241BE0284641464746FD
:10014000224600F02AF953465A46C01A914110D36C
:1001500011461846224600F011F92D1A67EB0108E6
:100160004F4622460120002100F008F917EB000954
:100170004E41201EA4F10104DFDC484631462A46E8
:100180004346BDE8F09F30B480EA010202F000452A
:1001900030F0004221F0004013D090B1C30DD40DD7
:1001A000C2F31601C0F31600E41A41F4000140F452
:1001B00000027D34914201D3641C00E04900002C10
:1001C00002DA30BC002070474FF400000023914257
:1001D00001D3891A034340084FEA4101F7D151B1D5
:1001E000914202D14FF0004105E002D24FF00101EF
:1001F00001E06FF0010103EBC450284430BC00F073
:10020000DCB8420005D0C0F3C7525242914201DC33
:100210000020704700EBC15070472DE9FE4F81EA86
:10022000030404F0004421F0004100944FF0000B5F
:1002300023F0004350EA01045ED052EA03045BD08D
:10024000C3F30A54C1F30A552C44A4F2F3340194C5
:10025000A0FB0254C1F3130141F48011C3F3130353
:1002600043F4801301FB024400FB034E840A970A07
:1002700044EA815447EA8357A4FB076802958D0A34
:1002800005FB07854FEA932C04FB0C542705029DC0
:100290004FEA065847EA1637B5EB08056EEB070C30
:1002A000870E920E47EA811742EA8312A7FB0201EA
:1002B000B6EB0B0164EB00042B0D43EA0C335E1824
:1002C00044EB1C50DA465146E7FB0201C5F3130428
:1002D0004FEA0B3343EA14534FEA0432019C43EADA
:1002E0000603A4F10C040294009CCDE900B400F0D4
:1002F000AAF803B0BDE8F08F00200146F9E7962385
:100300000022114600F062B80EB540F2334102916E
:100310000021CDE900110A460B4600F094F803B025
:1003200000BD20F00040C10DC0F3160040F40000F5
:100330007F2901DA00207047962903DCC1F196017C
:10034000C8407047963988407047C1F30A5210B5CB
:10035000C1F3130140F2FF3341F480119A4201DAF4
:10036000002010BD40F233439A42A2F2334203DC34
:10037000524200F012F810BD904010BD202A04DB5C
:10038000203A00FA02F1002070479140C2F12003A8
:1003900020FA03F3194390407047202A04DB203AE7
:1003A00021FA02F00021704721FA02F3D040C2F195
:1003B000200291400843194670470029A8BF7047A2
:1003C000401C490008BF20F00100704710B4B0FA8B
:1003D00080FC00FA0CF050EA010404BF10BC704726
:1003E00049B1CCF1200421FA04F411FA0CF118BF40
:1003F000012121430843A3EB0C01CB1D4FEA00610F
:100400004FEA102042BF002010BC704700EBC350E1
:1004100010440029A4BF10BC7047401C490008BF0D
:1004200020F0010010BC704710B5141E73F10004D9
:1004300008DA401C41F1000192185B411A4301D1D6
:1004400020F0010010BD2DE9F04D92469B4611B100
:10045000B1FA81F202E0B0FA80F220329046FFF762
:100460008DFF04460F4640EA0A0041EA0B0153465D
:100470005A46084313D0114653EA010019D0C8F177
:1004800040025046FFF789FF05460E465046594642
:100490004246FFF773FF084305D0012004E02046E1
:1004A0003946BDE8F08D0020054346EAE0762C434E
:1004B00037430A986305E40AA0EB08000022FD0A0E
:1004C00044EA47540A3002D500200146E9E7010515
:1004D00010196941DDE9084500196941BDE8F04D91
:1004E000A2E70000064C074D06E0E06840F001037B
:1004F00094E8070098471034AC42F6D3FFF7FAFDB2
:10050000202900084029000870B58C1810F8015BFC
:1005100015F0070301D110F8013B2A1106D110F89C
:10052000012B03E010F8016B01F8016B5B1EF9D1A0
:100530002B0705D40023521E0DD401F8013BFAE726
:1005400010F8013BCB1A921C03E013F8015B01F891
:10055000015B521EF9D5A142D8D3002070BD0029FD
:10056000816802D041F4A00101E021F4A001816082
:100570007047000070B50446284DC0074FF4007165
:10058000284602D000F044FE01E000F03FFE600883
:10059000234EC0074FF48041304602D000F038FEB1
:1005A00001E000F033FEA008C0074FF400413046E0
:1005B00002D000F02DFE01E000F028FEE008C007A8
:1005C0004FF48061284602D000F022FE01E000F0E6
:1005D0001DFE2009C0074FF40061284602D000F03C
:1005E00017FE01E000F012FE6009C0074FF48051D1
:1005F000284602D000F00CFE01E000F007FEA00942
:10060000C0074FF40051284603D0BDE8704000F009
:10061000FFBDBDE8704000F0F9BD0000000C0140D6
:1006200000100140FEE7C1B2000A40EA0120704715
:100630002DE9F84F0020ADF80000DFF834A14BF6AB
:10064000BF7648F280074A4D4A4C40F68F7848F60C
:100650000F7BDFF824910AF1440A31E00888474A09
:1006600010F00F00107034D0454901EB8001D1F833
:10067000002CADF80020BDF8002012040BD5D1F8F5
:10068000002C02EA0802C1F8002C3E4901EB800070
:1006900050F8040C8047BDF80000000610D537481C
:1006A0003749007801EB8001D1F8002C02EA0B02F7
:1006B000C1F8002C344901EB800050F8040C80474D
:1006C000DAF800004946A9F800000004C6D4BDE8E5
:1006D000F88F28682080208800F030006080208813
:1006E00000F4405020802868304080F4005080F0B2
:1006F0002000384328600888C006286815D400EA1E
:100700000B00286000F0A8FE26E02188890401D5AE
:1007100080F400506188C90626D46188890601D515
:1007200080F0200038432860D1E7ADF80000BDF824
:100730000000000506D5286800EA0800286001F0DE
:1007400025FB09E0BDF800000004B9D5286800EADF
:100750000800286000F0A8FF286821883040C904FC
:10076000D3D580F48050D0E780F01000D5E70000AA
:10077000005C00405E010020420000204C0100208F
:1007800000500040680000204C0000208100084814
:100790000844D0F8001C490409D5D0F8001C48F6DC
:1007A0008F7211404CF280021143C0F8001C704758
:1007B00000500040810008480844D0F8001C490659
:1007C00009D5D0F8001C48F68F72114048F2C002DB
:1007D0001143C0F8001C70470050004081000648DB
:1007E0000144D1F8000C48F68F62104048F28002B4
:1007F0001043C1F8000C70470050004070B5144819
:100800000068144900F0F80302268B7008784A78D3
:1008100000F04004C81C002582B97CB173B1067099
:1008200043700D4805700B490422C91C812001F05A
:100830002FFEBDE87040012001F018BA0670437029
:100840008570C570002AECD0521E4A70E9E700009E
:10085000080801403400002010000020174910B59E
:100860000A68918841BB062804D1117801F07F0104
:10087000012905D0117801F07F0121290AD01BE060
:100880009078222802D0212802D015E00C490CE0F3
:100890000C490AE0032802D009280DD101E00A49D9
:1008A00003E00B4B09490920187029B10020916120
:1008B00050828847002010BD022010BD500100204A
:1008C00015090008ED080008F9080008690A000881
:1008D00084000020014901F01FBB000094000020AB
:1008E000014901F019BB00008C000020014901F012
:1008F00013BB0000A400002008B10448704704495D
:10090000012009680882002070470000880000204C
:1009100050010020014901F0FFBA00009C000020B6
:1009200005490968C978042901D900207047034A9C
:1009300002EBC10101F0F0BA50010020DC00002000
:1009400009B9002800D00220704700000649096854
:10095000097801F07F01212901D10B2801D0022063
:10096000704700F075B8000050010020274810B50E
:10097000006800218172C1722549C9794172002045
:1009800001F05CF84FF40071002001F081F91021B2
:10099000002001F053F91821002001F0D7F8582168
:1009A000002001F02DF90020FFF718FF194890F8FA
:1009B0002C10002001F0DAF8002001F00FF94FF4BC
:1009C000C061012001F064F94FF48071012001F051
:1009D00017F94FF48271012001F0B8F804210120C9
:1009E00001F01EF90E21012001F0C0F84FF4405132
:1009F000012001F0DBF82021012001F01FF9002087
:100A000001F080F804490120086010BD5001002069
:100A1000F8270008AC0000202401002006480068E8
:100A2000807A002806D00549052008600121044885
:100A3000FFF795BD70470000500100202401002001
:100A4000002401400149042008607047240100206F
:100A5000034804490068C0784860002070470000DF
:100A6000500100208400002008B104487047044968
:100A7000022009680882002070470000D20100208F
:100A8000500100207047704710B500F0F1FB054899
:100A900000240068847200F05FFE01F0D7FC024879
:100AA000046010BD500100202401002070B51249DF
:100AB00007200870114C124D20682B680209A2EB28
:100AC0001312042A13D90F4E327882B10E4A1268DB
:100AD000052A0CD1000948700222812001F0D8FCBF
:100AE000012001F0C3F82068286000203070BDE8C4
:100AF0007040022000F00AB83401002000000020FD
:100B0000040000201000002024010020C10002D5B4
:100B10000249086070470249486070470404024077
:100B2000000002402DE9F047DFF89480254F4FF098
:100B30003009D8F8001001F11005088A0E7A08B9BA
:100B4000042E04D0AC88A04215D8042614E01E4818
:100B50000178012903D00726102038802BE01B4A9A
:100B6000002112681A4B120403EBD2325160A7F82D
:100B7000009001701FE00226844200D90446A96853
:100B8000204688478246002000F064FB014622464A
:100B9000504601F091FC2146002001F041F82888E0
:100BA000001B2880688820446880A7F800900949C5
:100BB0004FF440500880D8F800000672BDE8F08776
:100BC000500100206001002062010020505C0040C4
:100BD000006000405E0100202DE9F047224EDFF862
:100BE0008C803027356835F8100FA968A9B100B39B
:100BF000AC88844200D9044620468847814628882C
:100C0000001B2880688820446880002000F002FBD8
:100C100001462246484600F06BFD288848B1144939
:100C20004FF4405008800021084600F0F9FFA8F872
:100C300000702888A988884201D3032001E020B1F0
:100C4000052031680872BDE8F08731680620087217
:100C5000084900200968084A090402EBD1314860BC
:100C6000A8F80070EFE700005001002060010020AC
:100C70005E010020505C004000600040F8B55D4C13
:100C80005D4D09262068002729684278062A05D08C
:100C9000AAB1082A4DD00A2A50D06BE00278520639
:100CA00068D18078012804D0022804D0032804D019
:100CB00060E0C96956E0096A54E0496A52E0428836
:100CC000B2BBC288022A55D102798ABB0278530688
:100CD00001D1838833B102F07F02012A04D0022AB5
:100CE0000CD047E045493DE08A69407900219047B2
:100CF000F0B92068807A0028F4D13BE0417901F016
:100D00000F0001F070020B063D4901EB8001D1F8A4
:100D1000001C03D5C1F30111090102E0C1F3013147
:100D20000903384B1B78834224D90AB90029D9D149
:100D300020E0007840061DD1334913E0027802F02C
:100D40007F02012A16D1827AA2B1428892B9027931
:100D500082B9C288012A0DD18A6940790021904761
:100D600040B92A4931B12068478281610020884713
:100D7000002006E029682068096940788847032830
:100D800013D021680A8AA2F57F43FF3B0BD00228CB
:100D90000ED06AB10878000626D5C8880090824235
:100DA0000AD9088218E00E72F8BD20680672F8BDF4
:100DB0004FF008000872F8BD0ED22868144B90F866
:100DC0002C00824201D21F7006E0B2FBF0F400FB5F
:100DD000142008B901201870286890F82C00888227
:100DE000BDE8F840FFF79EBE0320087209490003E2
:100DF0000880F8BD50010020540100205D1F00084C
:100E000000500040FC000020F11E0008351F0008C3
:100E1000620100205E0100207047000001490120AE
:100E200008707047100000200449022048700449EF
:100E3000012008704FF4405100F0B8BE340000208B
:100E400011000020704700002DE9F0414FF40077B9
:100E5000384600F059F800281FD0114D2878A0B16D
:100E600010480068052810D10F4C2070022000F0B7
:100E7000D7FD002670B1667002220B49812001F077
:100E800007FB012000F0F2FE2E703846BDE8F0416D
:100E900000F00CB801206070EEE7BDE8F0810000C2
:100EA00010000020240100203401002001490860C6
:100EB00070470000140401407CB500208DF8040048
:100EC000102001248DF8050000948DF80640684636
:100ED00000F02AF80120FFF7E9FF022000906846A1
:100EE00000F022F80220FFF7E1FFA5042846FFF7F3
:100EF000DDFF08208DF8050000958DF80640684656
:100F000000F012F87CBD0000064A0146002012687D
:100F1000044B0A4014331B680B4202D0002A00D055
:100F2000012070470004014030B51A4983790268F6
:100F300053B30B6893430B600A1D13680468A34303
:100F4000136002790A441368046823431360114A4A
:100F5000083213680468A3431360131D1C680568F6
:100F6000AC431C604479102C05D021440A68006809
:100F700002430A6030BD116804682143116019689A
:100F800000680143196030BD00790844016891434D
:100F9000016030BD0004014070B504460C4DC0072F
:100FA0004FF40041284602D000F032F901E000F091
:100FB0002DF9A009C0074FF02001284603D0BDE855
:100FC000704000F025B9BDE8704000F01FB9000086
:100FD000000C014070B505464FF43026304600F055
:100FE00053F8042811D1094C206940F00200206117
:100FF0006561206940F040002061304600F044F80F
:10100000216941F6FD721140216170BD002002404E
:1010100008490420CA68D20701D001207047CA6875
:10102000520701D502207047C968C906FBD50320C5
:1010300070470000002002402DE9F84106460020DC
:101040004FF4005700900D46384600F01DF8042874
:1010500016D10C4C206940F0010020613580B84663
:10106000384600F011F8BF1E042806D1B61C280C23
:1010700000963080404600F007F821693940216130
:10108000BDE8F8810020024000B50346FFF7C0FF2D
:1010900003E000BFFFF7BCFF5B1E012803D0002B5D
:1010A00000D1052000BD002BF4D1FAE7F8B50121ED
:1010B000302000F07DFB0121042000F079FB0121AC
:1010C000082000F075FB0121102000F071FB2820A2
:1010D0008DF80300B020ADF800001D4D02248DF8FE
:1010E00002406946284600F039F848208DF8030090
:1010F0008020ADF800008DF802406946284600F0D7
:101100002DF810248DF803404FF47F40ADF8000017
:10111000104E01258DF802506946304600F01EF849
:101120008DF803404FF46040ADF800008DF8025098
:101130006946094800F012F88DF803402020ADF808
:1011400000008DF802506946304600F007F8F8BDFF
:1011500000080140000C014000100140F0B5CA78C1
:10116000002502F00F03D20601D58A7813430A78CE
:101170004FF00F0E12F0FF0F4FF001021CD0046869
:101180000F8802FA05F63740B74211D14FEA850CB5
:101190000EFA0CF724EA070703FA0CF43C43CF7865
:1011A000282F02D0482F02D002E0466100E00661FD
:1011B0006D1C082DE4D304600C88FF2C1ED94468F4
:1011C0005FF0000606F1080702FA07F50F882F40C6
:1011D000AF420FD14FEA860C0EFA0CF7BC4303FA6C
:1011E0000CF73C43CF78282F00D14561CF78482FAA
:1011F00000D10561761C082EE4D34460F0BD0246A0
:10120000002092680A4200D0012070474161704777
:10121000016170470549096889B201EBC0000449C2
:1012200001EB4000008980B270470000505C004034
:10123000006000400549096889B201EBC00004491B
:1012400001EB40008089C0F309007047505C00400A
:10125000006000400449096889B201EBC0000349FD
:1012600031F8100080B27047505C004000600040D0
:101270000A4810B50168001D0468001D00680818C0
:101280000BD00822064900F03BF90549204604220C
:10129000BDE81040103100F033B910BDE8F7FF1F72
:1012A0001A000020FEE7000010B5012186B04805B5
:1012B00000F072FA0121082000F07AFAC020ADF89F
:1012C000100003208DF812001C208DF8130004A9D3
:1012D0001048FFF743FF0020ADF804004BF6FF7005
:1012E000ADF806003820ADF808004FF48060ADF886
:1012F0000A000001ADF80C000748084C00900121DD
:10130000204600F00DF86946204600F03DF806B092
:1013100010BD0000000C0140A086010000540040F8
:101320000029018802D041F0010101E021F0010112
:10133000018070470029018802D041F4807101E0EA
:1013400021F48071018070470029018802D041F4A6
:10135000007101E021F40071018070470CB5024674
:10136000002000920A0F21F07F41019202D0009AE2
:10137000143202E0009A090C1832009212680A42F4
:1013800000D001200CBD000070B50446808886B0F6
:101390000D4620F03F06684600F016FA27490298ED
:1013A000B0FBF1F189B20E43A680228822F001023F
:1013B0002280234B2A689A421CD85200B0FBF2F0DC
:1013C00080B2042800D20420491C2184A0832088F4
:1013D00040F00100208021884FF6F5300140A888B8
:1013E0006A89104308432080A889298908432081FD
:1013F00006B070BDEB88A3F53F46FF3E0BD002EB75
:10140000C20303EB0212B0FBF2F080B240F4804062
:10141000020506D007E002EB4202B0FBF2F080B218
:10142000F6E740F001004FF4967251434FF47A72A0
:10143000B1FBF2F140F40040C6E7000040420F006B
:10144000A086010012B141F0010101E001F0FE01AE
:10145000018270470182704710B5134C2068017AF1
:10146000022904D0042902D0062905D015E0FFF78F
:1014700059FB2068007A11E04178052909D10178EB
:10148000490606D1C07800F03DFB08480068006AB4
:1014900080470748006880688047082021680872F4
:1014A000BDE8104000F036B950010020580100207E
:1014B0005401002010B50121042000F06DF90E4800
:1014C0004FF4FA610D4A0068B0FBF1F0401E108045
:1014D000101D018009481C38018841F0010101807C
:1014E00006482838018841F0010101804FF0E021D1
:1014F000C004C1F8000110BD3801002028080040D8
:10150000F0B500230A24302537261F4611E000BF1E
:10151000B4EB107F02D905EB107C01E006EB107CE8
:1015200001F813C001EB430C00015B1C8CF8017047
:10153000DBB29342ECD3F0BD0448817A044809B190
:10154000052100E00121016000F052BE00020020F0
:1015500024010020FEE770477047000070B50F239C
:10156000C47801780122F4B1144C2468457804F45D
:10157000E064C4F5E064240AC4F10406E34084781E
:10158000B5401C402C4301F1E021230181F80034D7
:10159000007800F01F018A404009800000F1E0203F
:1015A000C0F8002170BD01F01F0082404809800092
:1015B00000F1E020C0F8802170BD00000CED00E0DB
:1015C0000249084302490860704700000000FA051C
:1015D0000CED00E070B52F4D2868017844784A067C
:1015E00006D001F07F00012828D002282BD035E05A
:1015F000092C06D0052C07D0032C0ED0012C14D0BA
:101600002CE000F0F5FC28E0C1787F292ED8817805
:1016100061BB818851BB807A27E0C17801291DD147
:101620008088D8B900F000FD17E0C178012915D1F4
:10163000818899B9407A80060AD40FE00B2C0DD12D
:1016400000F048FD09E0012C02D0032C03D005E096
:1016500000F0D0FB01E000F0F9FC58B10E49204643
:10166000096849698847032802D018B108200DE0AD
:1016700009200BE0094A062000211268084B1204D9
:1016800003EBD2325160074A302111802968087279
:1016900070BD00005001002054010020505C00404B
:1016A000006000406001002010B50F4C2068007AF7
:1016B000022811D004280FD0032804D0052802D016
:1016C000072805D008E0FFF787FA2068007A04E0D1
:1016D00006480068C0688047082021680872BDE895
:1016E000104000F017B80000500100205401002005
:1016F000064B521C520803EB410105D031F8043B64
:1017000020F8023B521EF9D17047000000600040F3
:10171000704700000C4810B590F82C10002000F025
:1017200025FA0A480068007A082802D0092809D05A
:1017300006E007494FF480500880064910200880D1
:10174000002010BD012010BDAC0000205001002081
:101750005E0100206001002010B5012000F082FD34
:101760000648012101600021054A0160031D19603E
:101770004FF4E05111800160002010BD405C00403A
:101780005C010020034A516821F44041014351604B
:101790007047000000100240044A0029D16901D0BE
:1017A000014300E08143D161704700000010024016
:1017B000044A0029916901D0014300E0814391610D
:1017C000704700000010024030B51F494A6812F00F
:1017D0000C031E4A03D0042B01D0082B21D0026039
:1017E0004A680F231A4C03EA1212A35C0268DA401B
:1017F00042604B68072505EA1323E35C22FA03F3F2
:1018000083604B6805EAD323E35CDA40C260496831
:10181000032303EA9131231F595CB2FBF1F101610B
:1018200030BD4A684B6802F470124FF0020413F4A2
:10183000803F04EB924202D04B689B0301D5054BDD
:1018400000E0024B5A43CAE70010024000127A003F
:101850006A01002000093D000149C1F8D800704725
:10186000000042422DE9F041214C072800D02070B1
:1018700022781F4D0627052104261E48062A0BD272
:10188000DFE802F0030C11161E27686810B1217002
:10189000BDE8F08100F030F82770F9E700F02CF88F
:1018A0002670012022E00220607003202070EFE704
:1018B0006078401E607060780028E9D12670E7E704
:1018C000026892B242F01002026021700A20607039
:1018D000DEE76178491E617061780029D8D101681E
:1018E00089B221F010010160277000206860CFE705
:1018F0002C010020405C004010B5064C206880B2EE
:1019000020F004002060FFF717FE4FF43F402060F6
:1019100010BD0000405C00402DE9F84F394901201E
:1019200000F0A4FD374C384E4FF40051A0783070D1
:101930008009C207354802D0FFF76AFC01E0FFF7D3
:1019400065FC20796179000640EA0140A179E579DA
:1019500040EA01200543B06894F80390DFF8B0B086
:10196000B24685421ED04846FEF7CEFC0746884662
:101970002846FEF7C9FC6FF003025B46FEF74DFCFC
:1019800006463A4643460091FEF747FCFEF7DDFC6B
:1019900000F044FE30460099FEF7D7FC00F056F800
:1019A000CAF8085080211B48FFF729FCB8B9B9F1E3
:1019B000010F14D1E07AC00611D5174E3046FFF75B
:1019C00009FB2846FEF7A0FC6FF003025B46FEF71A
:1019D00024FCFEF7BAFC01463046FFF72DFB607889
:1019E000FFF7DAFAE07A4FF480410009C2070B48AA
:1019F00003D0BDE8F84FFFF70BBCBDE8F84FFFF789
:101A000005BC0000C401002034000020001001408B
:101A100083D7A73F00080140B0AE0008000C01408A
:101A20000349044A31F8101052F82000FFF7E7BBD1
:101A3000B0280008A401002070470000024920F0EF
:101A40000700086070470000505C004070B5044615
:101A50001E481F4D2044A84202D20120FEF78AFDF5
:101A60001C481D492044884202D20220FEF782FD14
:101A70001A481B492044884202D20420FEF77AFD0E
:101A8000184819492044884202D20820FEF772FD06
:101A900016482044A84202D21020FEF76BFD1448DD
:101AA00014492044884202D22020FEF763FD1248E8
:101AB000A4F5EA44313C844202D24020FEF75AFDAC
:101AC0000E4800680E49486070BD0000FFE448FF02
:101AD0009F2526005F9C90FF5FB74700BFB4B3FF10
:101AE0005F1823009FEFB7FE1FB381005FDAD9FFB5
:101AF0005FBF22FFBFCF6A006FB02500B0AE000805
:101B000008000020F0B50E490E4D48F68F770B788F
:101B1000002148F2800C0BE0CEB205EB8604D4F82D
:101B2000002C3A40324342EA0C02C4F8002C491C13
:101B30009942F1D3044940F080000860F0BD0000F4
:101B4000FC000020005000404C5C0040054A21F0A1
:101B50000101126892B202EBC000034A02EB40009E
:101B600081607047505C0040006000400D4A126880
:101B70003E2992B202EBC0000B4A02EB400209D9A7
:101B80004809C90601D1401E80B24FF4004141EA24
:101B9000802004E04808C90700D0401C8002106083
:101BA00070470000505C00400C60004082000A4812
:101BB0000244D2F8000C4BF68F731840CB0401D5C9
:101BC00080F48050890401D580F4005048F28001EF
:101BD0000843C2F8000C70470050004081000748DD
:101BE0000144D1F8000C4BF68F72104080F4405045
:101BF00048F280021043C1F8000C704700500040CA
:101C0000054A21F00101126892B202EBC000034ABA
:101C100042F8101070470000505C00400060004027
:101C2000044A126892B202EBC000034A02EB400081
:101C300041607047505C00400060004082000A48EC
:101C40000244D2F8000C48F6BF731840CB0601D509
:101C500080F01000890601D580F0200048F2800154
:101C60000843C2F8000C704700500040810007484C
:101C70000144D1F8000C48F6BF72104080F03000EB
:101C800048F280021043C1F8000C70470050004039
:101C9000820005480244D2F8000C48F68F13184021
:101CA0000843C2F8000C7047005000400CB50021FA
:101CB000264801910091026842F4803202604FF49C
:101CC000A063026802F400320092019A521C019251
:101CD000009A12B9019A9A42F3D10268920333D55D
:101CE000012100911A490A6842F010020A600A684C
:101CF00022F003020A600A6842F002020A604168A8
:101D0000416041684160416841F4806141604168DF
:101D100021F47C114160416841F4881141600168FF
:101D200041F08071016001688901FCD5416821F0B2
:101D300003014160416841F0020141604168C1F323
:101D400081010229FAD10CBD00910CBD00100240A6
:101D50000020024010B501212020FFF729FD4FF49B
:101D60004040FFF70FFDFFF7A1F9FFF79DFABDE82F
:101D70001040FFF7A1B810B50020FFF76DFD01215D
:101D8000BDE81040C805FFF707BD000070B5164854
:101D90000068174D0004C10B14480144098989B239
:101DA00000EB41042868017A09290FD021780170DD
:101DB00061784170A088FEF736FC29684880208948
:101DC000FEF731FC29688880A089C8802868012135
:101DD0000172C08828B1FEF751FFBDE87040FFF7DF
:101DE00099BCFFF7F7FBF8E7505C0040006000404B
:101DF000500100202DE9F04138480068017811F0C9
:101E00007F0102D0022905D066E0417A01F0DF01AE
:101E100041724EE0418800295ED10179F1BB4179E0
:101E2000304D21F080040A0605EB84022C4BD2F8D9
:101E3000002C03D5C2F30112120102E0C2F30132F9
:101E400012031E782346A64246D93AB3807A28B3B5
:101E500008064FEA84000ED52844D0F8000CC0F3E1
:101E60000110012821D11846FEF7A4FC204630219C
:101E7000FFF7E4FE19E04619D6F8000CC0F3013074
:101E8000012812D14BF68F7748F28008A4B118468A
:101E9000FEF77CFCD6F8000C384000E01CE080F433
:101EA000405040EA0800C6F8000C0F48006840693E
:101EB00080470020BDE8F0810C4890F82C100020ED
:101EC000FFF754FED5F8000C384080F4405040EA4B
:101ED0000800C5F8000CE8E70220EBE750010020FD
:101EE000FC0000200050004058010020AC00002001
:101EF00010B5074C30B1074800680068804720687B
:101F00000A3010BD216801200882002010BD0000A9
:101F10005001002058010020054A13685A8A10B168
:101F20000868104470478888801A1882002070471B
:101F30005001002010B5074C30B107480068806898
:101F4000804720680C3010BD2168012008820020E5
:101F500010BD00005001002058010020204910B59C
:101F6000096860B11F48002202800A7853060AD02F
:101F700002F07F02012A16D0022A16D001E00220C8
:101F80000882002010BD497A8A06027802D542F004
:101F9000020201E002F0FD0249060270D1B211D442
:101FA00001F0FE0110E00F4810BD4A791107130639
:101FB0000D4A02EB9161D1F8001C07D5C1F3011164
:101FC00006E0017841F00101017003E0C1F3013145
:101FD0000129F6D00548006800698047E3E7000062
:101FE00050010020640100200050004058010020F2
:101FF0000A4810B500680A4AC1785278914203D85D
:1020000082780AB982880AB1022010BD817205481F
:10201000006840688047002010BD0000500100208B
:10202000FC00002058010020064810B50068417AE5
:1020300041F02001417204480068C06980470020D7
:1020400010BD0000500100205801002070B51D484F
:102050001D4D0368597921F0800005EB80000C06C6
:10206000D0F8004C21F0800203D5C4F30114240100
:1020700002E0C4F301342403144D2D78954210D9A5
:102080005A8872B96CB19A7A5AB10906D0F8001C14
:1020900048F2800207D548F6BF73194081F010015D
:1020A00006E0022070BD4BF68F73194081F4805119
:1020B0001143C0F8001C0648006880698047002072
:1020C00070BD00005001002000500040FC000020C6
:1020D0005801002010B50E4C0E4A20681268C178D5
:1020E00092694079904721688A7A22B118B90879B3
:1020F00008B9887808B1022010BD07480068C06898
:10210000804720684179C172C1780173002010BDF9
:10211000500100205401002058010020F8B52B493F
:10212000002000900A682A4B2A4C92B203EB8005EB
:10213000D5F8005CADB244F82050401C0828F5D317
:1021400042F48060086040F00100086020F0010562
:102150000D601E4A121D10684005FCD54FF6FF3079
:102160001060002054F8206003EB8007B6B2C7F877
:10217000006C401C0828F5D345F00800086008688A
:1021800080B240F004000860134B18680090186893
:1021900020F0030040F0010018601048046844F08B
:1021A000040404601468E40401D430BF09E04EF66E
:1021B000FF7414600A6892B222F008020A60009963
:1021C0001960016821F004010160F8BD405C004025
:1021D00000500040E00100200070004010ED00E0E1
:1021E00002480168491E0160704700001400002089
:1021F0000F4810B5016841F00101016041680D4AC6
:102200001140416001680C4A11400160016821F4ED
:1022100080210160416821F4FE0141604FF41F01FB
:102220008160FFF743FD05494FF00060086010BD75
:10223000001002400000FFF8FFFFF6FE08ED00E08E
:102240000449012008700448018821F0010101803F
:102250007047000010000020100800404FF480205C
:10226000FEF724BE704700000648054902220160BF
:102270000A72064A0449C0E90112086800470000D2
:102280000002002050010020AC00002000010020CE
:1022900038B54FF4A060FFF793F914208DF80000D3
:1022A00001258DF8015000248DF802408DF803506F
:1022B0006846FFF753F92A208DF800008DF8014099
:1022C0008DF803506846FFF749F917208DF8000094
:1022D0008DF801406846FFF741F928208DF800008D
:1022E0008DF801406846FFF739F90B208DF80000A2
:1022F00002208DF801006846FFF730F938BD000074
:102300002DE9F0414A4E88B000243068494D68807C
:102310006888494F39880840000401D5FEF788F9DC
:10232000688839884FF6FF380840400504D5C6F85C
:1023300000804248406880476988388801408904A5
:1023400002D54DF6FF71316069880140C80405D59A
:102350004EF6FF7030600020FFF784FA68883988F5
:10236000084000050BD53648007810B1FFF7D6FEBF
:1023700002E00220FFF776FA4FF2FF7030606988C2
:1023800038880140890505D54FF6FF51316029781D
:10239000491C297069880140C80545D54FF6FF6082
:1023A00030602348001D00684FF00001000437D55D
:1023B0006868401C68606868032832D91C48001FA0
:1023C000026812072DD4026892B2AA601D4A6B46B9
:1023D00002EB8407D7F8007CBFB243F82470641C7A
:1023E000082CF5D3AC6844F00104AC60AC68A4B22E
:1023F0000460AC6824F00104AC60AC68A4B2046072
:1024000030684005FCD5C6F80080002053F8204015
:1024100002EB8006A4B2C6F8004C401C0828F5D395
:1024200069600720FFF71EFA08B0BDE8F0810000E0
:10243000445C0040400000205C010020AC00002013
:102440002801002000500040FFF75ABF0549002036
:10245000086005494FF43F4008800249091F0860A1
:1024600000207047445C00405C01002070B500F023
:102470007F060D463046FEF7DDFE04463046FEF789
:10248000C9FE014622462846FFF732F9204670BDB4
:1024900070B500F07F0514460E462846FEF7DAFEBA
:1024A0000146A2B2304600F007F8A1B22846FFF775
:1024B000B7FB002070BDFEE7094B10B5521C520857
:1024C00003EB41010AD000BF10F8013B521E10F887
:1024D000014B43EA042321F8043BF5D110BD000071
:1024E0000060004002E008C8121F08C1002AFAD1AB
:1024F00070477047002001E001C1121F002AFBD184
:102500007047000070B50F4C054601212046FEF7CC
:1025100011FF0D4E20463146FEF720FF0028F9D06E
:10252000E9B200222046FEF78DFF074D6D1C2946BB
:102530002046FEF713FF0028F9D002481830008823
:1025400070BD00000054004001000010012101484E
:10255000FEF7FABE0054004070B50A4C0146204612
:10256000FEF778FF084E084D7C3E29462046FEF7D0
:10257000F5FE0028F9D031462046FEF7EFFE002890
:10258000F3D070BD0054004080000010FFF7E2FB64
:10259000FFF77EFEFFF7EFFBFFF766FEFEF78AFF11
:1025A0000D480C4941600D49416000F01FF80C4D89
:1025B0000C4C0D4F0126607808B1FFF7ADF9286883
:1025C0000528F8D120780028F5D03E80FEF716F9CE
:1025D000F1E700002301674500200240AB89EFCD01
:1025E00024010020100000202408004010B5D22152
:1025F000B72000F069F82021B12000F065F84F21E4
:10260000102000F061F88021B12000F05DF86F210A
:10261000BDE81040112000F057B8000070B5014629
:10262000002000F015F8094D0446287810B16878AC
:1026300084420AD02021B12000F046F84F2110201A
:1026400000F042F8012028706C7070BD0800002076
:102650002DE9F0470646184842681848B0FBF1F4E7
:10266000E00700D0641E04FB01F0B0FBF2F1CDB234
:10267000B0FBF2F102FB1100DFF8449000214B4661
:10268000A0FB03788C4601FB098100FB0C11384646
:102690000023FDF747FD02460A484B462946805D68
:1026A00000F058F807480022801C2146805D00F0A9
:1026B0001BF82846BDE8F087080000200046C32329
:1026C000FFFF0F00E227000870B504460D46C0204A
:1026D000FFF718FF2046FFF73FFF2846FFF73CFFB4
:1026E000BDE87040FFF732BF2DE9F04107461848BA
:1026F0000D4600EBC5141646C020FFF703FF384611
:10270000FFF72AFF0020FFF727FF0120FFF724FF34
:10271000C4F301403043042D17D000210843FFF7D4
:102720001BFFC4F30720FFF717FFE0B2FFF714FF0A
:102730000020FFF711FF0020FFF70EFF0020FFF73A
:102740000BFFBDE8F041FFF701BF0C21E6E70000F9
:1027500000FEFFFF2DE9F041804616460D461C465F
:102760001846FDF7CCFD07463046FDF7C8FD394653
:10277000FDF709FD0721FDF744FDFDF7D2FD00EB54
:10278000C5156043C0EBC616C020A5F50075FFF760
:10279000B9FE4046FFF7E0FEC4F30720FFF7DCFE7A
:1027A000E0B2FFF7D9FEC5F30140FFF7D5FEC5F350
:1027B0000720FFF7D1FEE8B2FFF7CEFEF02000EAD7
:1027C0001430C6F303410843FFF7C6FEC6F30720E3
:1027D000FFF7C2FEF0B2FFF7BFFEBDE8F041FFF722
:1027E000B5BE1A222A321201000200000040830402
:1027F000505700020102030109022900010100E013
:102800003209040000020300000009211001000148
:1028100022300007058103040001070501030E00B3
:10282000010600FF0901A10185010901150025012B
:102830007508950DB1828501090191828502090211
:102840001500250175089503B18285020902818270
:10285000C0040309040A03520061004A0061001623
:102860000352004800490044002000530054004D2A
:10287000003300320000000000022000000440008D
:102880004000800000010002004000000000020043
:1028900004000000200000000400000020000000F0
:1028A00010000000100000001000000010000000E8
:1028B00001000020000201000200000100400010A1
:1028C00004000000100000000800000040000000AC
:1028D0004000000020000000200000002000000058
:1028E0000100002000020100020000010040001071
:1028F00000000200010004000400030003000300C4
:1029000000000D0009000000010008000E000C008E
:1029100006002800170006000700170028002800FE
:102920004029000800000020C4010000080500083C
:10293000F8290008C40100205C040000F424000809
:1029400001107201141A03521248122D3A30020279
:102950002531131D0E0C14085915040A19291C8160
:1029600013E6273308121AF80832291321283308EE
:10297000301A0A08320913890A14086D091B0885E0
:10298000081A8704135D081B084D101A41041AE148
:102990000C1AD5041A210C4132401A513832041A4B
:1029A0005508320A1A5F083216221833201A1A0202
:1029B000ED29801A1D4C09169C1A451C41192BE162
:1029C0002BA24A5B513F010203040607A301174CE7
:1029D00002040646192A992E143801401A44AB1AEB
:1029E00008081A14046908DA1004291829081A0CAE
:0829F000045A180429285904B7
:04000005080000ED02
:00000001FF
